S032000052414D436F646556325F4154393153414D394732302D454B5F44617461466C61736836344D4269745F4C452E6D6F7401
S11300008700C1004B01A902150331043D0400001F
S113001010B4BD4A10608020800053680342FCD0B5
S1130020FF230C0C1C40146054680442FCD00C0ADE
S11300301C40146054680442FCD00B4013605168A7
S11300400142FCD010BC7047F8B5B04C80273F018A
S113005067600021A160AE4DD7216960BE08A96820
S11300603142FCD000F0EAF98020FF216960AA68DF
S11300703242FCD0AA68D207FCD52A680242F5D0E5
S11300802760A760F1BD10B4516801220468012300
S1130090A34000240C808B70CC700A714A718C715F
S11300A0CA710A724C728A720A614C610469E41062
S11300B08C61806882409818C000C86110BC704789
S11300C0F3B581B057685469012001990968012387
S11300D08B400199896888401B1810690021984257
S11300E02ED2029A00231360884D802212016A6086
S11300F0AB60019A1268521C914001430B20FFF738
S113010087FF834EFF207060B0688005FCD501989E
S113011000F094F9FF207060B0688005FCD5B068E9
S1130120C007FCD5306838707F1C641EF2D1802073
S113013000012860A86002980021416003B0F0BD6E
S1130140491CC01A9842CCD3FAE7F1B584B0506880
S113015001900120049B1B6898400123049CA4681F
S1130160A340C0180090546916690027864250D2F3
S113017000200860654D002E02D1009884424DD2C3
S11301808020000168600020A8603900049800689D
S1130190401C81405320FFF73BFF80200001286072
S11301A0A8600498FFF750FF8020000168600020D9
S11301B0A86031008420FFF72BFF0098861BA6421D
S11301C000D92600A41B049800F038F9019800789F
S11301D00199491C01914C49086048688005FCD587
S11301E0761EF3D1802000012860A860686000209A
S11301F0A860390004980068401C81408820FFF7FB
S113020007FF802000012860A8600498FFF71CFF06
S113021043E07F1C361A8642AAD3FAE7019802907B
S11302208020000168600020A86000218420FFF77E
S1130230EFFE01200499096888400121049A92681C
S113024091404618049800F0F9F802980078029951
S1130250491C02912C49086048688005FCD5761E2B
S1130260F3D1802000012860A860029801908020CA
S1130270000168600020A860390004980068401CF0
S113028081408820FFF7C4FE802000012860A86018
S11302900498FFF7D9FE0098241A7F1C0026002C2E
S11302A000D06AE705B0F0BDF1B50120009B1B68E2
S11302B001249C40009B9B6898402018C00013694F
S11302C0002683421AD2546900200860002C14D0FE
S11302D00E4D80273F016F600020A8603100009818
S11302E0C06881405020FFF793FE2F60AF600098F4
S11302F0FFF7AAFE761C641EEAD1F1BD761C1B1A18
S11303008342E0D3FAE700000C80FCFF30F8FFFFE3
S11303100880FCFF30B44D494D4A0A604D4907221C
S11303200A604A610A674A60802109014A4A1160E9
S11303304A4B1960116391631161494B80241C601D
S11303401C60484C5C60484C5C6301241C60516335
S113035000249463D724DC608C081D692542FCD0FA
S1130360FF25DD601D692542FCD01D69ED07FCD524
S11303709B68116391639A101207120FD21E120622
S11303800AD0520E062A51D801A39B5C9F44C04652
S1130390081E364C58708800082101600B2141600A
S11303A0032181600D21C160046130BC70470821C4
S11303B001600B214160032181600D21C160610056
S11303C0016130BC7047082202600B2242600322A4
S11303D082600C22C260016130BC70470821016058
S11303E00B214160032104E0092101600C214160DB
S11303F0042181600D21C160E100016130BC7047BE
S1130400092101600C214160042181600D21C1603A
S11304102101016130BC70470A2101600D21416056
S1130420052181600E21C1602101016130BC70474A
S11304300021016041608160016170470B4841689F
S1130440090401D40A4901607047000010FCFFFF51
S11304501410000000F4FFFF00F8FFFFA0F8FFFFF6
S11304600080FCFF110001000A03010040FDFFFFB2
S1070470010000A5DE
S9030000FC
